:100000000C945E000C9486000C9486000C94860080
:100010000C9486000C9486000C9486000C94860048
:100020000C9486000C9486000C9486000C94860038
:100030000C9486000C9486000C9486000C94860028
:100040000C9466020C9486000C94D6020C94B002B8
:100050000C9486000C9486000C9486000C94860008
:100060000C9486000C9486000000000024002700F9
:100070002A0000000000250028002B0004040404CE
:100080000404040402020202020203030303030342
:10009000010204081020408001020408102001021F
:1000A00004081020000000080002010000030407FB
:1000B000000000000000000008034A0511241FBED4
:1000C000CFEFD8E0DEBFCDBF22E0ACEAB1E001C0A7
:1000D0001D92AF35B207E1F711E0A0E0B1E0EEE12B
:1000E000FFE002C005900D92AC3AB107D9F710E0DD
:1000F000CDE5D0E004C02197FE010E948A05CC35F1
:10010000D107C9F70E9493030C9482070C94000056
:10011000E9EAF0E02491E5E9F0E09491E1E8F0E02B
:10012000E491EE23C9F0222339F0233001F1A8F441
:10013000213019F1223029F1F0E0EE0FFF1FEE58C7
:10014000FF4FA591B4912FB7F894EC91811126C07F
:1001500090959E239C932FBF08952730A9F02830B7
:10016000C9F0243049F7209180002F7D03C02091F1
:1001700080002F7720938000DFCF24B52F7724BD18
:10018000DBCF24B52F7DFBCF2091B0002F772093BC
:10019000B000D2CF2091B0002F7DF9CF9E2BDACFC7
:1001A0003FB7F8948091B4019091B501A091B60148
:1001B000B091B70126B5A89B05C02F3F19F0019655
:1001C000A11DB11D3FBFBA2FA92F982F8827BC01B1
:1001D000CD01620F711D811D911D42E0660F771FD9
:1001E000881F991F4A95D1F708958F929F92AF92D9
:1001F000BF92CF92DF92EF92FF926B017C010E943F
:10020000D0004B015C01C114D104E104F104B9F048
:100210000E94D000681979098A099B09683E7340D9
:100220008105910580F321E0C21AD108E108F108A7
:1002300088EE880E83E0981EA11CB11CE4CFFF90CD
:10024000EF90DF90CF90BF90AF909F908F900895E8
:10025000AF92BF92CF92DF92EF92FF920F931F93D4
:10026000CF93DF936C017B018B01040F151FEB0112
:100270005E01AE18BF08C017D10759F06991D601C9
:10028000ED91FC910190F081E02DC6010995892B3B
:1002900079F7C501DF91CF911F910F91FF90EF90FA
:1002A000DF90CF90BF90AF900895FC01538D448DA7
:1002B000252F30E0842F90E0821B930B541710F011
:1002C000CF96089501970895FC01918D828D98171E
:1002D00061F0A28DAE0FBF2FB11D5D968C91928DF6
:1002E0009F5F9F73928F90E008958FEF9FEF089527
:1002F000FC01918D828D981731F0828DE80FF11DF0
:10030000858D90E008958FEF9FEF0895FC01918D0A
:10031000228D892F90E0805C9F4F821B91098F7303
:100320009927089588EB91E00E94860121E0892BAE
:1003300009F420E0822F089580E090E0892B29F0D5
:100340000E94920181110C9400000895FC01A48D7B
:10035000A80FB92FB11DA35ABF4F2C91848D90E0E7
:1003600001968F739927848FA689B7892C93A089CA
:10037000B1898C91837080648C93938D848D981354
:1003800006C00288F389E02D80818F7D80830895E7
:10039000EF92FF920F931F93CF93DF93EC0181E0D5
:1003A000888F9B8D8C8D98131AC0E889F98980817C
:1003B00085FF15C09FB7F894EE89FF896083E889AF
:1003C000F98980818370806480839FBF81E090E0A1
:1003D000DF91CF911F910F91FF90EF900895F62E2E
:1003E0000B8D10E00F5F1F4F0F731127E02E8C8DC8
:1003F0008E110CC00FB607FCFACFE889F98980810D
:1004000085FFF5CFCE010E94A601F1CFEB8DEC0F59
:10041000FD2FF11DE35AFF4FF0829FB7F8940B8F29
:10042000EA89FB8980818062CFCFCF93DF93EC0193
:10043000888D8823B9F0AA89BB89E889F9898C91CC
:1004400085FD03C0808186FD0DC00FB607FCF7CF88
:100450008C9185FFF2CF808185FFEDCFCE010E9488
:10046000A601E9CFDF91CF91089581E00E94880035
:100470006CE370E080E090E00E94F50080E00E9474
:10048000880064E170E080E090E00C94F50081E089
:100490000E94880064E170E080E090E00E94F50036
:1004A00080E00E94880064E170E080E090E00C94BD
:1004B000F500FC0101900020E9F73197AF01481BDE
:1004C000590BBC0188EB91E00C9428011F920F920C
:1004D0000FB60F9211242F933F938F939F93AF9357
:1004E000BF938091B0019091B101A091B201B09100
:1004F000B3013091AF0123E0230F2D3758F501965A
:10050000A11DB11D2093AF018093B0019093B10163
:10051000A093B201B093B3018091B4019091B50161
:10052000A091B601B091B7010196A11DB11D8093B4
:10053000B4019093B501A093B601B093B701BF91F8
:10054000AF919F918F913F912F910F900FBE0F9080
:100550001F90189526E8230F0296A11DB11DD2CF3A
:100560001F920F920FB60F9211242F933F934F9328
:100570005F936F937F938F939F93AF93BF93EF930B
:10058000FF9388EB91E00E94A601FF91EF91BF914C
:10059000AF919F918F917F916F915F914F913F911B
:1005A0002F910F900FBE0F901F9018951F920F92D2
:1005B0000FB60F9211242F938F939F93EF93FF9376
:1005C000E091C801F091C9018081E091CE01F091E4
:1005D000CF0182FD1BC090818091D1018F5F8F730D
:1005E0002091D201821741F0E091D101F0E0E8546E
:1005F000FE4F958F8093D101FF91EF919F918F9145
:100600002F910F900FBE0F901F9018958081F4CFFF
:100610001092BB011092BA0188EE93E0A0E0B0E026
:100620008093BC019093BD01A093BE01B093BF0124
:100630008AE091E09093B9018093B80185EC90E055
:100640009093C5018093C40184EC90E09093C7011E
:100650008093C60180EC90E09093C9018093C8011B
:1006600081EC90E09093CB018093CA0182EC90E002
:100670009093CD018093CC0186EC90E09093CF01D4
:100680008093CE011092D1011092D2011092D30129
:100690001092D401109256021092550210925802F4
:1006A0001092570210925A021092590264E270E0BE
:1006B00090E080E00E94B506009701F19093560209
:1006C0008093550223E230E0309358022093570282
:1006D0002091590230915A02232B11F4FC0110820F
:1006E00083E290E090935A028093590268E171E0AE
:1006F00080915502909156020C947B07809155028F
:1007000090915602009711F00E942C06109256020A
:100710001092550210925A021092590210925802E9
:10072000109257020895789484B5826084BD84B590
:10073000816084BD85B5826085BD85B5816085BDDC
:1007400080916E00816080936E0010928100809194
:10075000810082608093810080918100816080931C
:100760008100809180008160809380008091B10041
:1007700084608093B1008091B00081608093B0006C
:1007800080917A00846080937A0080917A00826000
:1007900080937A0080917A00816080937A008091C2
:1007A0007A00806880937A001092C100E091C801BD
:1007B000F091C90182E08083E091C401F091C5010C
:1007C0001082E091C601F091C7018FEC80831092F6
:1007D000D001E091CC01F091CD0186E08083E091E1
:1007E000CA01F091CB01808180618083E091CA01D0
:1007F000F091CB01808188608083E091CA01F09103
:10080000CB01808180688083E091CA01F091CB01A7
:1008100080818F7D8083E5E9F0E02491E1E8F0E0DC
:100820008491882399F090E0880F991FFC01E85982
:10083000FF4FA591B491FC01EE58FF4F8591949123
:100840008FB7F894EC91E22BEC938FBF80E4D82E15
:1008500000E010E0D0927C0080917A008064809368
:100860007A0080917A0086FDFCCF8091780090918B
:100870007900883E9340C4F48CE391E00E945902D1
:1008800087E591E00E94590260ED77E080E090E01A
:100890000E94F50001151105E9F20E9492018823DA
:1008A000C9F20E940000D6CF8AE591E00E94590269
:1008B00087E591E00E94590264EF71E080E090E0EA
:1008C0000E94F500E0905902F0905A02F092AE01B9
:1008D000E092AD01D0E0C0E0CE15DF050CF0D5C050
:1008E0008091590290915A02C817D90720F01092AE
:1008F000AC012196F1CF809155029091560200975C
:10090000B1F38C0F9D1FFC0180818093AC01823676
:1009100009F50E94350264E170E080E090E00E94F9
:10092000F5000E94470264E170E080E090E00E94E0
:10093000F5000E94470264E170E080E090E00E94D0
:10094000F5000E94470264E170E080E090E00E94C0
:10095000F500CFCF833659F40E94350264E170E090
:1009600080E090E00E94F5000E94470209C08436B2
:1009700019F40E943502D7CF873649F40E94350218
:1009800064E170E080E090E00E94F5001AC08B36D0
:1009900059F40E94350264E170E080E090E00E942A
:1009A000F5000E9447023BC08C3649F40E94470282
:1009B00064E170E080E090E00E94F500DACF8E36CE
:1009C00019F40E943502B7CF823771F2863759F495
:1009D0000E94470264E170E080E090E00E94F50030
:1009E0000E944702D8CF803319F50E94350264E196
:1009F00070E080E090E00E94F5000E94350264E122
:100A000070E080E090E00E94F5000E94350264E111
:100A100070E080E090E00E94F5000E94350264E101
:100A200070E080E090E00E94F5000E9435028BCFDC
:100A3000813319F40E944702DACF833399F40E947C
:100A4000470264E170E080E090E00E94F5000E94BF
:100A5000470264E170E080E090E00E94F5000E94AF
:100A60004702D5CF843349F40E94470264E170E025
:100A700080E090E00E94F500ABCF803209F039CFE2
:100A80006CE370E080E090E062CF68EB7BE080E0B8
:100A900090E0FECE8091550290915602009711F0A1
:100AA0000C942C0608952F923F924F925F926F9272
:100AB0007F928F929F92AF92BF92CF92DF92EF92EE
:100AC000FF920F931F93CF93DF93CDB7DEB7CA1B6F
:100AD000DB0B0FB6F894DEBF0FBECDBF09942A889A
:100AE000398848885F846E847D848C849B84AA8442
:100AF000B984C884DF80EE80FD800C811B81AA81CF
:100B0000B981CE0FD11D0FB6F894DEBF0FBECDBF99
:100B1000ED010895EE0FFF1F0590F491E02D09946B
:100B20000F931F93CF93DF938230910510F482E0EF
:100B300090E0E0915D02F0915E0230E020E0B0E0F4
:100B4000A0E0309799F42115310509F44AC0281B1B
:100B5000390B24303105D8F58A819B8161157105E7
:100B600089F1FB0193838283FE0111C04081518191
:100B70000281138148175907E0F04817590799F483
:100B8000109761F012960C93129713961C9332965D
:100B9000CF01DF91CF911F910F91089500935D02D6
:100BA00010935E02F4CF2115310551F0421753071F
:100BB00038F0A901DB019A01BD01DF01F801C1CFC5
:100BC000EF01F9CF90935E0280935D02CDCFFE01DD
:100BD000E20FF31F819391932250310939832883C7
:100BE000D7CF20915B0230915C02232B41F42091FE
:100BF00002013091030130935C0220935B0220914B
:100C00000001309101012115310541F42DB73EB7A6
:100C10004091040150910501241B350BE0915B02CA
:100C2000F0915C02E217F307A0F42E1B3F0B28178C
:100C3000390778F0AC014E5F5F4F2417350748F055
:100C40004E0F5F1F50935C0240935B028193919320
:100C50009FCFF0E0E0E09CCFCF93DF930097E9F0E7
:100C6000FC01329713821282A0915D02B0915E0264
:100C7000ED0130E020E01097A1F420813181820F56
:100C8000931F20915B0230915C022817390709F00D
:100C900061C0F0935C02E0935B02DF91CF91089515
:100CA000EA01CE17DF07E8F54A815B819E01411515
:100CB0005105B1F7E901FB83EA8349915991C40FCA
:100CC000D51FEC17FD0761F4808191810296840F96
:100CD000951FE90199838883828193819B838A830D
:100CE000F0E0E0E012968D919C9113970097B9F592
:100CF0002D913C911197CD010296820F931F209167
:100D00005B0230915C022817390739F6309751F5AC
:100D100010925E0210925D02B0935C02A0935B029F
:100D2000BCCFD383C28340815181840F951FC817E4
:100D3000D90761F44E5F5F4F88819981480F591F31
:100D4000518340838A819B8193838283211531055E
:100D500009F0B0CFF0935E02E0935D029ECFFD01FB
:100D6000DC01C0CF13821282D7CFB0E0A0E0EBEB62
:100D7000F6E00C9455058C01009751F4CB010E94CC
:100D800090058C01C801CDB7DEB7E0E10C94710588
:100D9000FC01E60FF71F9C0122503109E217F3070F
:100DA00008F49DC0D901CD91DC911197C617D707E2
:100DB00098F0C530D10530F3CE0104978617970718
:100DC00008F3C61BD70B2297C193D1936D937C93E5
:100DD000CF010E942C06D6CF5B01AC1ABD0A4C0194
:100DE0008C0E9D1EA0915D02B0915E02512C412C93
:100DF000F12CE12C109731F580915B0290915C020F
:100E00008815990509F05CC04616570608F058C0C9
:100E10008091000190910101009741F48DB79EB738
:100E20004091040150910501841B950BE817F907C7
:100E300008F055C0F0935C02E0935B02F901718306
:100E40006083A0CF8D919C91119712966C90129710
:100E500013967C901397A815B90559F56C0142E0DB
:100E6000C40ED11CCA14DB0420F1AC014A195B0981
:100E7000DA011296159780F0628273825183408363
:100E8000D9016D937C93E114F10471F0D7011396AD
:100E9000FC93EE93129776CF22968C0F9D1FF9014B
:100EA00091838083F301EFCFF0935E02E0935D02C4
:100EB00069CF4816590608F42C017D01D3019ACF59
:100EC000CB010E9490057C01009749F0AE01B8016A
:100ED0000E947207C8010E942C06870153CF10E0C0
:100EE00000E050CFFB01DC0102C001900D924150A7
:100EF0005040D8F70895FB01DC0101900D920020CD
:100F0000E1F7089510E0CDE5D0E004C0FE010E94B5
:0E0F10008A052196CE35D107C9F7F894FFCF98
:100F1E0000005F02800000000000C801280155019A
:100F2E00150286016401780131206220722033207F
:100F3E0034206B2063203020642033203420342072
:100F4E006C203120762031206E2067006E6565643E
:100F5E00203556206F6E20416E616C6F676963207D
:100F6E00706F72742030000D0A0036382031303523
:100F7E002031303320313035203131362039372091
:100F8E00313038203332203131322031303520317A
:100F9E003130203332203533203332203131372077
:100FAE003131302031303820313131203939203152
:0C0FBE003037203130312031303000005D
:00000001FF
